:020000040800F2
:1000000000040020E1010008E3010008E30100080A
:10001000E3010008E3010008E3010008E301000830
:10002000E3010008E3010008E3010008F9250008E6
:10003000E3010008E3010008E3010008E301000810
:10004000E3010008E3010008E3010008E301000800
:10005000E3010008E301000849370008753700088C
:10006000A1370008CD370008F9370008E301000880
:10007000E3010008E3010008E3010008E3010008D0
:10008000E3010008E3010008E3010008E3010008C0
:10009000E3010008E3010008E30100082538000837
:1000A000E3010008E3010008E3010008E3010008A0
:1000B00065350008E3010008E3010008E3010008DA
:1000C000E3010008E3010008E3010008E301000880
:1000D000E3010008990F0008AD0F0008E3010008D4
:1000E0008D380008E3010008E3010008E30100087F
:1000F000E3010008E3010008E3010008E301000850
:10010000E3010008E3010008E3010008E30100083F
:10011000E3010008C10F0008E3010008E301000843
:10012000E3010008E3010008E3010008E30100081F
:10013000E3010008E3010008E3010008E30100080F
:10014000E3010008E3010008E3010008E52C0008D2
:10015000E3010008E3010008E3010008E3010008EF
:10016000E3010008E3010008E3010008E3010008DF
:10017000E3010008E3010008E3010008E3010008CF
:10018000E3010008E3010008E3010008E3010008BF
:10019000E3010008E3010008E3010008E3010008AF
:1001A000E3010008E3010008E3010008E30100089F
:1001B000E3010008E3010008E3010008E30100088F
:1001C000E3010008E3010008E3010008E30100087F
:1001D000E3010008E3010008E3010008E30100086F
:1001E00002E000F000F8FEE772B6394880F30888B4
:1001F000384880F3098838484EF60851CEF200019D
:10020000086040F20000CCF200004EF63471CEF2ED
:1002100000010860BFF34F8FBFF36F8F40F2000003
:10022000C0F2F0004EF68851CEF200010860BFF334
:100230004F8FBFF36F8F4FF00000E1EE100A4EF6C4
:100240003C71CEF200010860062080F31488BFF3F1
:100250006F8F02F00FFA03F01BF94FF055301F4972
:100260001B4A91423CBF41F8040BFAE71C49194A6A
:1002700091423CBF41F8040BFAE71A491A4A1B4B5A
:100280009A423EBF51F8040B42F8040BF8E70020F5
:100290001749184A91423CBF41F8040BFAE702F0B3
:1002A000EDF903F051F9144C144DAC4203DA54F853
:1002B000041B8847F9E700F03FF8114C114DAC42A0
:1002C00003DA54F8041B8847F9E702F0D5B90000B7
:1002D000000400200024002000000008000000208E
:1002E00000040020083D00080024002028240020ED
:1002F0002824002060410020E0010008E0010008FF
:10030000E0010008E00100082DE9F04F2DED108A12
:10031000C1F80CD0C3689D46BDEC108ABDE8F08FD3
:10032000002383F311882846A047002001F026FE11
:1003300001F0D6FD00DFFEE71A4B6FF0780270B5D2
:1003400000241A700F225C709C70DC701C715C7150
:100350009C71DC711C725C729A72DC7202F01AF988
:10036000064602F043F9054650B90F4B9E4217D09E
:1003700001339E4241F2883412BF05460024012514
:10038000002002F00DF90DB100F0B4F800F002FD0C
:1003900000F0E4FB204600F00BF900F0ABF8F9E7C1
:1003A0000446EDE728240020010007B008B500F05E
:1003B00053FBA0F120035842584108BD07B5054B37
:1003C00002211B88ADF8043001A800F0B1FB03B096
:1003D0005DF804FB8C390008064991F8243033B1EC
:1003E00000230822086A81F8243000F0D9BB0120DC
:1003F000704700BF482400202DE9F84F234C94F8A3
:1004000024300546884617468BBB2E46DFF87C9085
:10041000002F38D094F824A0BAF1000F05D1202283
:10042000FF214846266200F0A3FCCAF10805BD4240
:1004300028BF3D465FFA85FBAD0041462A4604EBE6
:100440008A0000F06BFC94F82430A7EB0B079B4468
:100450005FFA8BFBBBF1080F2E44A844FFB284F86F
:1004600024B0D5D1FFF7B8FF0028D1D108E0266A23
:1004700006EB8306B042C9D0FFF7AEFF0028C4D117
:100480000020BDE8F88F0120BDE8F88F4824002047
:1004900010B5202383F311881248C3680BB101F013
:1004A000F3FD0023104A0F484FF47A7101F0B0FDBC
:1004B000002383F311880D4C236813B12368013B9B
:1004C0002360636813B16368013B6360084B1B786A
:1004D00033B9636823B9022000F016FC322363604D
:1004E00010BD00BF342400209104000878290020AA
:1004F0007024002010B5254B254953F8042F0132F4
:1005000000D110BD8B42F8D1224C234B22689A4275
:100510003AD9224B9B6803F1006303F580339A427A
:1005200032D2002000F034FB1D4B0220187000F086
:10053000E1FB1C4B1A6C00221A64196E1A66196EC4
:10054000596C5A64596E5A665A6E5A6942F0800262
:100550005A615A6922F080025A615A691A6942F056
:1005600000521A611A6922F000521A611B6972B6B0
:100570000D4A0E4B13601B682268202181F31188FD
:100580009D4683F30888104710BD00BFFCFF00089C
:100590001C00010804000108FFFF000828240020B7
:1005A000702400200038024008ED00E0000001083F
:1005B0002DE9F04FB54C97B020228246FF210EA8BE
:1005C000A56800F0D5FBB24A1378A046A3B9B1489C
:1005D0000121C3601170202383F31188C3680BB11C
:1005E00001F052FD0023AC4AAA484FF47A7101F0A1
:1005F0000FFD002383F31188DFF8BCB2BAF1000FBE
:1006000001D0CBF800A0A54F00243C70CBF80440EB
:100610002646012000F06EFBBAF1000F00F0E081E9
:10062000DBF80030002B40F0DB8117B0BDE8F08F25
:100630000220FFF7BBFE002840F0D081984B1B88BA
:10064000ADF82430022109A800F072FAE1E74FF476
:100650007A7000F001FA031E0193EFDB0220FFF72E
:10066000A5FE81460028E9D0019B581E0428E5D844
:10067000DFE800F0030C0F12150016A8052340F860
:10068000343D042100F054FA4C4650E004217F48E8
:10069000F8E704218348F5E704218348F2E71C24A6
:1006A000204600F077FA04340990042109A800F0EC
:1006B0003FFA2C2CF4D1E7E7002EBFD0002CBDD0A0
:1006C0000220FFF773FE064610B901242646B5E75F
:1006D000012000F05DFA0220387000F00BFB0024CE
:1006E000E3B21846019300F063FA814648B1019BDA
:1006F000184600F06DFA01340028F1D134466B4BF6
:100700009DE7012302203B7000F0EAFA4D46D8F83D
:1007100008309D4206D2284600F03CFA0130EDD167
:100720000435F4E700253D70CBF80450344600F062
:1007300027FBFFF743FE4EE1002E3FF47FAF002C76
:100740003FF47CAF0220387000F0D4FA322000F081
:1007500083F9041EB9DB14F00306B6D1D8F80820DB
:100760002B199342B1D8B4F5807FAED8DFF8409111
:10077000A6420CDA4FF47A7000F06EF90390039BF6
:10078000002BA2DB039B06F809300136F0E7C820F6
:10079000FFF70CFE0646002897D01F2D11D8C5F193
:1007A0002009A14528BFA1460EAB25F003004A460B
:1007B0003F49184400F0B2FA4A46FF213C4800F095
:1007C000D7FA4FEAA4095FFA89F239492846FFF7B8
:1007D00013FE0446002891D005EB89050646A6E7DE
:1007E0000220FFF7E3FD00283FF428AFFFF7F4FDF8
:1007F00000283FF423AF4FF0000AD146D8F8083064
:100800009A453CD2BAF11F0F1CD80E9B013319D068
:100810002AF0030316AA134453F8203C09932549F0
:100820004B68A3B1002209A8135C83EA0903DBB279
:10083000013251F82330042A83EA1929F4D10AF14C
:10084000040ADBE7504600F0A5F90990E7E71A46ED
:10085000082012F0010F4FEA52021FBF82F06D42D2
:1008600082F4380282F4034282F020020138F0D18F
:1008700041F823200133B3F5807FE8D1D2E716A8F1
:10088000042140F8489D00F053F950E72824002047
:1008900074250020342400209104000870240020D6
:1008A0008E3900082C2400203024002090390008C4
:1008B00074240020782500207829002016A8002321
:1008C00040F8343D642100F0FFF800287FF4B6AE14
:1008D0000220FFF76BFD00283FF4B0AE099800F04E
:1008E00089F916AB43F8440D04211846CBE716A846
:1008F000002340F8343D642100F0E6F800287FF43E
:100900009DAE0220FFF752FD00283FF497AE0998F4
:1009100000F07EF916AB43F8400DE5E70220FFF743
:1009200045FD00283FF48AAE00F078F916AB43F895
:100930003C0DD9E70220FFF739FD00283FF47EAED9
:1009400009A9142000F070F9814616A8042140F886
:10095000389D00F0EDF8494609A894E74FF47A7005
:10096000FFF724FD00283FF469AEFFF735FD0028AE
:100970003FF4C5AE0E9B01330CD008220EA9002017
:10098000FFF73AFD00283FF4BAAE2022FF210EA85F
:1009900000F0EEF9FFF712FD2E4801F0F5FA44E6FB
:1009A00016A8002340F8343D642100F08DF800289B
:1009B0007FF444AE0220FFF7F9FC00283FF43EAE7E
:1009C000FFF7FCFC41F2883001F0DEFA099800F0F4
:1009D0001FFA00F0D5F94FF0000A1AE60646A6E61F
:1009E000002000F039F80390039B002BFFF614AEB3
:1009F000012000F075F9039B213B122B3FF609AE55
:100A000001A252F823F000BF310600084F0600088B
:100A1000B9060008130600081306000813060008AC
:100A20003907000813060008E1070008BD080008A0
:100A3000EF0800081D090008130600083509000822
:100A4000130600085D0900082F07000813060008B8
:100A5000A1090008A08601002DE9F34702AE002499
:100A60004FF47A7506F8014D144FDFF8588045436E
:100A700097F900305A1C5FFA84F901D0A34212D1D1
:100A800058F8240003680122D3F820A031462B46F1
:100A9000D047012807D10A4B9DF8070083F8009042
:100AA00002B0BDE8F0870134042CE1D14FF4FA70B4
:100AB00001F06AFA4FF0FF30F2E700BF0024002097
:100AC00098290020D03900082DE9F0474FF47A75B5
:100AD000144FDFF8588006464D43002497F9003044
:100AE0005A1C5FFA84F901D0A34210D158F82400AF
:100AF00003680422D3F820A031462B46D0470428AF
:100B000005D1094B83F800900020BDE8F08701343F
:100B1000042CE3D14FF4FA7001F036FA4FF0FF30B5
:100B2000BDE8F0870024002098290020D039000873
:100B300030B4074B1A78074B53F822402368DD691D
:100B4000054B0A46AC460146204630BC604700BF14
:100B500098290020D0390008A086010070B501F066
:100B60005BFC094C094E20700025306823788342D5
:100B700008D901F04BFC336805440133B5F5803FDB
:100B80003360F2D370BD00BF992900208029002076
:100B900001F0ECBC00F1006000F5803000687047A7
:100BA00000F10060920000F5803001F077BC000099
:100BB000054B1A68054B1B789B1A834202D91044D7
:100BC00001F024BC002070478029002099290020D2
:100BD00038B5074D04462868204401F01FFC28B9A9
:100BE00028682044BDE8384001F030BC38BD00BF63
:100BF0008029002010F0030308D1B0F5007F05D84C
:100C000000F10050A0F508400068704700207047D0
:100C1000014BC058704700BF107AFF1F014B186886
:100C2000704700BF002004E070B52A4B1C68C4F375
:100C30000B03240C63B140F21342934231D040F2D3
:100C4000194293422FD040F2214293422DD10323E7
:100C5000214A0C2505FB03235D6893F9082042F225
:100C600001039C4224D0B4F5805F23D041F20103FC
:100C70009C4221D041F203039C421FD041F2070362
:100C80009C4208BF3122441E0C44013D0B46A34246
:100C90001ED215F9016F581C96B1034600F8016C7D
:100CA000F5E70123D4E70223D2E73F220B4DD6E735
:100CB0003322E3E74122E1E75A22E4E75922E2E75F
:100CC0002C2584421D7001D9981C5A70401A70BDA1
:100CD0001846FBE7002004E0A0390008943900081A
:100CE000022802BF024B4FF080629A61704700BF3A
:100CF00000080240022802BF024B4FF480629A6152
:100D0000704700BF00080240022801BF024A536931
:100D100083F48063536170470008024010B50023DC
:100D2000934203D0CC5CC4540133F9E710BD0000FA
:100D300030B5441E14F9010F0B4660B193F9005011
:100D4000854201F1010106D11AB993F90020801AF8
:100D500030BD013AEEE7002AF7D1104630BD000061
:100D600002460346981A13F9011B0029FAD170476D
:100D700002440346934202D003F8011BFAE770478E
:100D8000024B1A78024B1A70704700BF9829002056
:100D900000240020F8B5184C1848194D194E174F6B
:100DA00000F03AFC2146154800F062FC2368164822
:100DB0005A6DD2F8043843F00203C2F8043801F047
:100DC000E3F82068114900F05FFD23685A6DD2F8FE
:100DD000043823F00203C2F804384FF4E1332B60E7
:100DE000002456F82400B84202D0294600F072FBD5
:100DF0000134042CF5D1F8BDB83A000814370020AE
:100E000084290020D039000840420F00083B000828
:100E100038B50B4B1A780B4B53F822400A4B9C42C7
:100E200005460CD0094B002118461422FFF7A0FFFD
:100E3000056001462046BDE8384000F04BBB38BD98
:100E400098290020D0390008143700208429002078
:100E5000026843681143016003B1184770470000FE
:100E6000024AD36843F0C003D360704700100140CA
:100E7000024AD36843F0C003D36070470044004087
:100E8000024AD36843F0C003D3607047005000406B
:100E90002DE9F041D0F85C64F7683368DA0505465F
:100EA0009CB20DD5202383F311884FF400710430D8
:100EB000FFF7CEFF6FF480733360002383F3118854
:100EC000202383F3118805F1040814F02F0333D194
:100ED00083F31188380615D5210613D5202383F313
:100EE000118805F1380000F053FA002846DA08218D
:100EF000281DFFF7ADFF4FF67F733B40F3600023E3
:100F000083F311887A060ED563060CD5202383F36C
:100F10001188EA6C2B6D9A4202D12B6C002B2FD1D9
:100F2000002383F31188D5F86424D368002B31D0D3
:100F30001069BDE8F0411847230713D014F0080FDB
:100F40000CBF00218021E00748BF41F02001A2072B
:100F500048BF41F04001630748BF41F480714046FB
:100F6000FFF776FFA406736805D595F86014284648
:100F7000194000F0BDFA3468A4B2A6E77060BEE77D
:100F800027F040073F041021281D3F0CFFF760FFAA
:100F9000F760C5E7BDE8F08108B50348FFF778FFC3
:100FA000BDE8084001F038BB9C29002008B5034883
:100FB000FFF76EFFBDE8084001F02EBB042E0020B5
:100FC00008B50348FFF764FFBDE8084001F024BB03
:100FD0006C32002010B50E4C0E4A2046002100F065
:100FE00057FA0D4BC4F85C340C4C0D4A20460021D6
:100FF00000F04EFA0B4BC4F85C340B4C0B4A00214A
:10100000204600F045FA0A4BC4F85C3410BD00BF1E
:101010009C290020610E000800100140042E0020D1
:10102000710E0008004400406C320020810E000860
:101030000050004038B5394D037C002918BF0D46DB
:10104000012B0446C0F8645410D1354B984242D16C
:10105000344B5A6C42F010025A645A6E42F010023D
:101060005A665B6E0B21252000F06AF82E4BD4F8EF
:101070005C249A422B6802D02C498A424BD12C49DD
:1010800001EB5301B1FBF3F3A988080442BF23F03D
:10109000070003F0070343EA40039360EB8843F043
:1010A00040039BB213612B8943F001039BB2536150
:1010B00041F4045343F02C03D36001F4A051002306
:1010C0001360B1F5806F136853680CBF7F23FF2353
:1010D00084F8603438BD174B98420CD1114B1A6C10
:1010E00042F400321A641A6E42F400321A661B6E21
:1010F0000B212620B8E7104B9842B7D1094B1A6C48
:1011000042F480121A641A6E42F480121A661B6E40
:101110000B213520A8E70949B2E700BF003A0008D3
:101120009C290020003802400010014000140140BA
:1011300000BD0105042E00206C32002080DE8002FC
:1011400000F1604300F01F02400903F5614309010B
:101150008000C9B200F1604083F8001300F56140DF
:1011600001239340C0F8803103607047F8B51546FD
:1011700082680669AA420B46816938BF8568761A7B
:10118000B542044607D218462A46FFF7C7FDA369B1
:101190002B44A3610DE011D932461846FFF7BEFD7E
:1011A000AF1B3A46E1683044FFF7B8FDE2683A44C5
:1011B000A261A3685B1BA3602846F8BD18462A46B7
:1011C000FFF7ACFDE368E4E783682DE9F0410446EE
:1011D00093421546266938BF85684069361AB5427C
:1011E0000F4606D22A46FFF799FD63692B446361D7
:1011F0000DE012D93246A5EB0608FFF78FFD4246F7
:10120000B919E068FFF78AFDE26842446261A368A9
:101210005B1BA3602846BDE8F0812A46FFF77EFDF0
:10122000E368E4E710B50A440024C361029B006050
:1012300040608460C160816141610261036210BDF0
:1012400008B582694369934201D1826882B9826894
:10125000013282605A1C42611970426903699A42E4
:1012600001D3C3684361002100F0AAFE002008BD3D
:101270004FF0FF3008BD000070B5202304460E4635
:1012800083F31188A568A5B1A368A269013BA36097
:10129000531CA36115782269934224BFE368A361BC
:1012A000E3690BB120469847002383F31188284651
:1012B00070BD3146204600F073FE0028E2DA85F367
:1012C000118870BD2DE9F74F05460F4690469A46A6
:1012D000D0F81C90202686F311884FF0000B14469E
:1012E00064B1224639462846FFF740FF034668B9F5
:1012F0005146284600F054FE0028F1D0002383F325
:101300001188A8EB040003B0BDE8F08FB9F1000F1D
:1013100003D001902846C847019B8BF31188E41A3B
:101320001F4486F31188DBE7C16081614161C361BD
:101330001144009B0060406082600161036270475D
:10134000F8B504460E461746202383F31188A56896
:10135000A5B1A368013BA36063695A1C62611E705A
:10136000236962699A4224BFE3686361E3690BB150
:1013700020469847002080F31188F8BD3946204662
:1013800000F00EFE0028E2DA85F31188F8BD0000B7
:10139000836942699A4210B501D182687AB982683C
:1013A000013282605A1C82611C7803699A4201D31F
:1013B000C3688361002100F003FE204610BD4FF09A
:1013C000FF3010BD2DE9F74F05460F4690469A466F
:1013D000D0F81C90202686F311884FF0000B14469D
:1013E00064B1224639462846FFF7EEFE034668B947
:1013F0005146284600F0D4FD0028F1D0002383F3A5
:101400001188A8EB040003B0BDE8F08FB9F1000F1C
:1014100003D001902846C847019B8BF31188E41A3A
:101420001F4486F31188DBE70268436811430160BB
:1014300003B11847704700001430FFF743BF0000A6
:101440004FF0FF331430FFF73DBF00003830FFF797
:10145000B9BF00004FF0FF333830FFF7B3BF0000D3
:101460001430FFF709BF00004FF0FF311430FFF7D1
:1014700003BF00003830FFF763BF00004FF0FF32BA
:101480003830FFF75DBF000000207047FFF7A2BDB6
:1014900037B50F4B0360002343608360C3600123B3
:1014A00004460374154600900B464FF4007200F199
:1014B0005C011430FFF7B6FE00942B464FF4007227
:1014C00004F5177104F13800FFF72EFF03B030BDAB
:1014D000143A000810B52023044683F31188FFF75F
:1014E000A9FD02232374002383F3118810BD00009B
:1014F00038B5C36904460D461BB904210844FFF7FB
:1015000093FF294604F11400FFF79AFE002806DA3B
:10151000201D4FF48061BDE83840FFF785BF38BD1E
:10152000026843681143016003B118477047000027
:1015300013B5446BD4F894341A681178042915D182
:10154000217C022912D11979128901238B4013427F
:101550000CD101A904F14C0001F014FED4F894441C
:10156000019B21790246206800F0DAF902B010BD33
:10157000143001F097BD00004FF0FF33143001F03C
:1015800091BD00004C3001F069BE00004FF0FF3308
:101590004C3001F063BE0000143001F065BD000066
:1015A0004FF0FF31143001F05FBD00004C3001F00E
:1015B00035BE00004FF0FF324C3001F02FBE00006E
:1015C000D0F8942438B5136819780429054601D059
:1015D000012038BD017C0229FAD112795C890120F1
:1015E00090400440F4D105F1140001F0F7FC0246EC
:1015F0000028EDD0D5F894544FF4807328686979A9
:1016000000F07CF9204638BD406BFFF7D9BF0000E1
:1016100000207047704700007FB5124B0360002325
:1016200043608360C360012502260F4B05740446A6
:101630000290019300F18402294600964FF48073D2
:10164000143001F0A7FC094B0193029400964FF46B
:10165000807304F52372294604F14C0001F06EFDFD
:1016600004B070BD3C3A00080916000831150008A6
:101670000B68202282F311880A7903EB82029061C1
:101680004A79093243F822008A7912B103EB8203C6
:10169000986102230374C0F89414002383F3118823
:1016A0007047000038B5037F044613B190F85430FA
:1016B000ABB9201D01250221FFF732FF04F1140010
:1016C00025776FF0010100F087FC84F8545004F195
:1016D0004C006FF00101BDE8384000F07DBC38BD22
:1016E00010B5012104460430FFF71AFF00232377C9
:1016F00084F8543010BD000038B50446002514307D
:1017000001F060FC04F14C00257701F02FFD201D55
:1017100084F854500121FFF703FF2046BDE838400C
:10172000FFF74EBF90F8443003F06003202B19D12F
:1017300090F84520212A0AD0222A4FF000030ED02B
:10174000202A0FD1084A82630722C26304E0064BB5
:1017500083630723C363002303640120704783630B
:10176000C363F9E70020704701240020D0F89434C7
:1017700037B51A681178042904461AD1017C022968
:1017800017D11979128901238B40134211D100F12D
:101790004C05284601F0AAFD58B101A9284601F0E0
:1017A000F1FCD4F89444019B21790246206800F0B2
:1017B000B7F803B030BD000000EB8103F7B59C69BA
:1017C00005460E46F4B1202383F3118805EB860706
:1017D000201D0821FFF7A4FEFB685B691B684C34E1
:1017E00013B1204601F0DCFC01A9204601F0CAFC3F
:1017F000024648B1019B3146284600F091F800238B
:1018000083F3118803B0F0BDFB685A691268002A9F
:10181000F5D01B8A013B1340F1D105F14402EAE700
:10182000093138B550F82140DCB1202383F3118809
:10183000D4F894241368527903EB8203DB689B6924
:101840005D6845B104216018FFF76AFE294604F17E
:10185000140001F0CDFB2046FFF7B2FE002383F316
:10186000118838BD7047000000F08EBF012303705F
:1018700000234360C36183620362C3624362036304
:10188000038143817047000038B50446202383F369
:10189000118800254160C56005614561856100F0E2
:1018A00083FF0223237085F3118838BD70B500EBE8
:1018B000810305465069DA600E46144618B11022BD
:1018C0000021FFF755FAA06918B110220021FFF797
:1018D0004FFA31462846BDE8704001F02FB80000AD
:1018E000028902F001020281428902F00102428172
:1018F000002202614261826101F0B4B8F0B400EBF1
:1019000081044789E4680125A4698D403D434581F0
:1019100023600023A2606360F0BC01F0CFB8000038
:10192000F0B400EB81040789E468012564698D4007
:101930003D43058123600023A2606360F0BC01F099
:1019400049B9000070B50223002504460370A0F8D1
:101950004C5080F84E5080F84F5005814581C5604D
:1019600005614561856180F8345000F083FF63684C
:101970001B6823B129462046BDE87040184770BD5A
:10198000436802781B6880F85020052202700BB172
:101990000421184770470000436890F850201B68E6
:1019A00002700BB1052118477047000090F83430E1
:1019B00070B5044613B1002380F8343004F14402BA
:1019C000204601F071F863689B6863BB94F844504B
:1019D00015F0600615D194F8453005F07F0545EA0D
:1019E000032540F202339D4200F00E815BD8022DA8
:1019F00000F0DC803FD8002D00F08780012D00F042
:101A0000CF800021204601F0A7FA0021204601F0F6
:101A100099FA63681B6813B106212046984706238C
:101A200084F8343070BD204698470028CED094F812
:101A30004B2094F84A3043EA0223E26B934238BFCA
:101A4000E36394F94430E56B002B4FF0200380F200
:101A5000FD80002D00F0EC80092284F8342083F30F
:101A600011880021E36BA26B2046FFF759FF00238A
:101A700083F3118870BDB5F5817F00F0B180B5F5B5
:101A8000407F49D0B5F5807FBBD194F84630012B1B
:101A9000B7D1B4F84C3023F00203A4F84C30A6635D
:101AA000E6632664C3E740F201639D421ED8B5F5A4
:101AB000C06F3BD2B5F5A06FA3D1B4F84430B3F5F5
:101AC000A06F0ED194F8463084F84E30204600F0D6
:101AD00029FF63681B6813B101212046984703233F
:101AE00023700023A363E3632364A0E7B5F5106FBD
:101AF00032D040F602439D4252D0B5F5006F80D1FE
:101B000004F14F03A363012324E004F14C03A36316
:101B10000223E36325648AE794F84630012B7FF4BF
:101B200070AFB4F84C3043F00203B6E794F84920A4
:101B3000616894F848304D6894F8471043EA0223EE
:101B4000204694F84620A84700283FF45AAF43683F
:101B5000A3630368E363A4E72378042B10D1202355
:101B600083F311882046FFF7BBFE86F31188636874
:101B700084F84F601B68032121700BB12046984701
:101B800094F84630002BACD084F84F3004232370F7
:101B900063681B68002BA4D0022120469847A0E769
:101BA000374BA3630223E36300239DE794F84810B7
:101BB00011F0800F204601F00F010ED000F066FFFB
:101BC000012806D002287FF41CAF2E4BA363E063EC
:101BD00067E72D4BA363E56363E700F049FFEFE799
:101BE00094F84630002B7FF40CAF94F8483013F093
:101BF0000F013FF476AF1A06204602D501F0C0F976
:101C00006FE701F0B3F96CE794F84630002B7FF4EE
:101C1000F8AE94F8483013F00F013FF462AF1B06A2
:101C2000204602D501F098F95BE701F08BF958E7FF
:101C3000142284F8342083F311882B462A4629463F
:101C40002046FFF75BFE85F3118870BD5DB115225C
:101C500084F8342083F311880021E36BA26B2046C3
:101C6000FFF74CFE03E70B2284F8342083F311883E
:101C70002B462A4629462046FFF752FEE3E700BFDF
:101C80006C3A0008643A0008683A000838B590F8E1
:101C900034300446152B29D8DFE803F03E282828E5
:101CA00028283E28280B29392828282828282828A9
:101CB0003E3E90F84B1090F84A20C36B42EA012256
:101CC0009A4214D9C268128AB3FBF2F502FB1535A9
:101CD0006DB9202383F311882B462A462946FFF746
:101CE0001FFE85F311880A2384F8343038BD14238D
:101CF00084F83430202383F3118800231A461946D0
:101D00002046FFF7FBFD002383F3118838BD036CE9
:101D100003B198470023E7E7002101F01DF90021F6
:101D2000204601F00FF963681B6813B106212046B5
:101D300098470623D8E7000090F83420152A38B5D4
:101D4000044622D80123934040F6416213421DD13C
:101D500013F480150FD19B0217D50B2380F8343074
:101D6000202383F311882B462A462946FFF7D8FD06
:101D700085F3118838BDC3689B695B682BB9036C18
:101D800003B19847002384F8343038BD002101F0B6
:101D9000E3F80021204601F0D5F863681B6813B111
:101DA0000621204698470623EDE70000024B00225B
:101DB0001B605B609A607047D43600200023037478
:101DC0008268054B1B6899689142FBD25A68036090
:101DD0004260106058607047D436002008B5202358
:101DE00083F31188037C032B05D0042B0DD02BB972
:101DF00083F3118808BD436900221A604FF0FF3356
:101E00004361FFF7DBFF0023F2E790E80C001A6064
:101E100002685360F2E70000002303748268054BF8
:101E20001B6899689142FBD85A6803604260106051
:101E300058607047D4360020054B1969087418683B
:101E400002681A605360186101230374FEF75CBADC
:101E5000D436002030B54B1C87B005460A4C10D054
:101E600023690A4A01A800F0D3F82846FFF7E4FFE7
:101E7000049B13B101A800F007F92369586907B062
:101E800030BDFFF7D9FFF8E7D4360020DD1D00088C
:101E900038B50C4D41612B6981689A6891420446BE
:101EA00003D8BDE83840FFF789BF1846FFF786FF23
:101EB00001232C61014623742046BDE83840FEF71B
:101EC00023BA00BFD4360020044B1A681B699068FF
:101ED0009B68984294BF002001207047D4360020B0
:101EE00010B5084C236820691A68226054600122EA
:101EF00023611A74FFF790FF01462069BDE8104086
:101F0000FEF702BAD4360020826002220274002258
:101F1000427470478368A3F17C0243F80C2C026979
:101F200043F83C2C426943F8382C074A43F81C2CF0
:101F3000C26843F8102C022203F8082C002203F890
:101F4000072CA3F1180070472103000810B52023C7
:101F500083F31188FFF7DEFF00210446FFF798FFA7
:101F6000002383F31188204610BD0000024B1B693B
:101F700058610F20FFF760BFD4360020202383F381
:101F80001188FFF7F3BF000008B50146202383F353
:101F900011880820FFF75EFF002383F3118808BD36
:101FA00049B1064B42681B6918605A601360436070
:101FB0000420FFF74FBF4FF0FF307047D4360020AA
:101FC0000368984206D01A6802605060596118464A
:101FD000FFF7F4BE7047000038B504460D46206890
:101FE000844200D138BD036823605C604561FFF71F
:101FF000E5FEF4E7054B03F114025A619A614FF0D4
:10200000FF32DA6100221A62704700BFD436002026
:10201000F8B503614FF08043C2605C6A194B1A4601
:10202000022952F8145F38BF0221954206461F4626
:102030000AD1586198611C62056045608160081989
:10204000BDE8F84001F074B9186AAB68241A0C199D
:1020500002D3E41A2D6804E09C4202D2204401F02D
:1020600075F9AB689C42F4D86B68736035601E608C
:102070006E60B460A9684FF0FF33091BA960FB6173
:10208000F8BD00BFD436002010B41B4C234653F8D3
:10209000141F814210D0416802680A6002685160D2
:1020A0009A424FF00001C16003D0936881680B44ED
:1020B00093605DF8044B70470A68626100209A42A1
:1020C0005360C86003D15DF8044B01F039B99368DF
:1020D0008868034493604FF08042206A526A121A63
:1020E0009342E6D9991A012998BF931C18445DF8C8
:1020F000044B01F02BB900BFD436002000207047FC
:10210000FEE70000704700004FF0FF30704700000E
:10211000022906D0032906D00129064818BF00204D
:10212000704705487047032A9ABF044800EBC20075
:1021300000207047643B0008183B0008082400207A
:1021400070B5044608460D46FEF70AFEC6B22046A4
:10215000013403780BB9184670BD32462946FEF7A4
:10216000E7FD0028F3D1012070BD00002DE9F04FFC
:1021700081469BB008460C461646FEF7F1FD3C49E9
:10218000C5B22046FFF7DCFF08B10535EDB239498D
:102190002046FFF7D5FF08B11035EDB2632D01AF32
:1021A0000CD8DFF8DCA0DFF8DCB03D4694F8008006
:1021B000B8F1000F1CD185F8008003E021463846B5
:1021C00001F0DCFB3846FEF7CBFDC0B2431C5B00E0
:1021D00089E84800337003237370002302361946E0
:1021E000DAB2904206F102063AD81BB0BDE8F08F91
:1021F000B8F1250F2FD107221D492046FEF798FD83
:1022000058B9DBF800202A60DBF804206A60DBF8AC
:102210000820AA6007340C35C8E708221549204673
:10222000FEF786FDB8B91448AA1C10F8011F134B1D
:102230004FEA111E01F00F011EF80AE011F80A1012
:1022400002F802EC984202F8011C02F10202ECD101
:1022500018350834AAE785F8008001340135A5E770
:10226000FA5C06F8022C06F8011C0133B8E700BF3F
:10227000C03A0008C83A00080F7AFF1F1B7AFF1FF8
:10228000DE3A0008D13A000808B5202383F311880C
:102290000348FFF76BFA002383F3118808BD00BFE2
:1022A0001437002010B50446052916D8DFE801F0E0
:1022B00016150316161D202383F311880E4A0121DB
:1022C000FFF7F4FA20460D4A0221FFF7EFFA0C4817
:1022D000FFF712FA002383F3118810BD202383F344
:1022E00011880748FFF7DEF9F4E7202383F311880C
:1022F0000348FFF7F5F9EDE7703A0008943A000853
:102300001437002038B50C4D0C4C0D492A4604F109
:102310000800FFF72BFF05F1CA0204F1100009497C
:10232000FFF724FF05F5CA7204F118000649BDE85D
:102330003840FFF71BBF00BFDC3B00200824002013
:10234000F03A0008FA3A0008C83A0008BFF34F8F85
:10235000024AD368DB03FCD4704700BF003C024054
:1023600008B5094B1B7873B9FFF7F0FF074B1A69E3
:10237000002ABFBF064A5A6002F188325A601A68C2
:1023800022F480621A6008BD3A3E0020003C024000
:102390002301674508B50B4B1B7893B9FFF7D6FFB0
:1023A000094B1A6942F000421A611A6842F48052DD
:1023B0001A601A6822F480521A601A6842F4806225
:1023C0001A6008BD3A3E0020003C02400B2870B560
:1023D00013D80B4A0B4C137863B90B4E4FF00061C6
:1023E00044F8231056F8235001330C2B2944F7D11D
:1023F0000123137054F8200070BD002070BD00BF91
:102400006C3E00203C3E0020843B0008014B53F80A
:1024100020007047843B00080C2070470B2810B543
:10242000044601D9002010BDFFF7D0FF064B53F83A
:1024300024301844C21A0BB9012010BD12680132B1
:10244000F0D1043BF6E700BF843B00080B2810B531
:1024500004461ED8FFF77AFFFFF782FF0E49F323E9
:10246000CB60FFF773FFC300DBB243F4007343F0AC
:1024700002030B610B6943F480330B61FFF766FFC6
:10248000FFF7A4FFFFF786FF2046BDE81040FFF7E7
:10249000C5BF002010BD00BF003C02402DE9F8433D
:1024A00012F00103154643D10244B2F1016F3FD24D
:1024B0002C4B1B6813F001033AD02B4CFFF750FF55
:1024C000F323E360FFF742FF40F20127032D16D804
:1024D000254C0F46401A40F20118EB1B0B44012B10
:1024E00000EB0706236926D823F001032361FFF7D9
:1024F00051FF0120BDE8F883043D0430E6E783077F
:10250000E6D1236923F44073236123693B432361AC
:1025100051F8046B0660BFF34F8FFFF717FF036896
:102520009E42E9D0236923F001032361FFF732FFC4
:102530000020BDE8F88323F440732361236943EA54
:1025400008032361B94637F8023B3380BFF34F8F4E
:10255000FFF7FCFE3688B9F80030B6B2B342BCD003
:10256000E0E700BF00380240003C0240084908B5DF
:102570000B7828B153B9FFF7F3FE01230B7008BDA8
:1025800023B1BDE808400870FFF704BF08BD00BFD5
:102590003A3E0020014B186D704700BF00280040F4
:1025A000094B1A6F120407D41A6F42F400721A67AB
:1025B0001A6F42F400421A67044A136843F48073A6
:1025C0001360034B186570470038024000700040EC
:1025D00000280040034B1B689B0042BF024B0122B6
:1025E0001A707047743802406D3E0020014B187815
:1025F000704700BF6D3E0020064A536823F0010378
:102600005360EFF30983683383F30988002383F36E
:102610001188704730EF00E010B5202383F3118854
:10262000104B5B6813F4006318D0F1EE103AEFF32F
:1026300009844FF0807344F84C3C0B4BDB6844F842
:10264000083CA4F1680383F30988FFF73DFC18B147
:10265000064B44F8503C10BD054BFAE783F3118854
:1026600010BD00BF00ED00E030EF00E031030008D6
:102670003403000870470000FEE70000084A094BD9
:1026800009498B4204D3094A0021934205D370477C
:1026900052F8040F43F8040BF3E743F8041BF4E784
:1026A0002C3D000860410020604100206041002076
:1026B000836D30B500229D68446D11464FF0FF30A8
:1026C00004EB421301329542C3F80019C3F8101904
:1026D000C3F80809C3F8001BC3F8101BC3F8080BA4
:1026E000EED24FF00113C4F81C3830BD890141F01F
:1026F0002001016103699B06FCD4122000F0AEBEEC
:10270000204B03EB80022DE9F047D2F80CE05D6D21
:10271000DEF81420461CD2F800C005EB063605EBA7
:102720004018516861450BD3D5F83428012303FACA
:1027300000F022EA0000C5F834081846BDE8F0872A
:10274000BEF81040ACEB0103A34228BF2346D8F8E3
:102750001849A4B2B3EB840F10D894681F46A4F1B3
:10276000040959F804AFC6F800A0042F01D9043FAA
:10277000F7E71C440B4494605360D2E70020BDE8A7
:10278000F08700BF703E002010B5054C2046FFF7D3
:102790006DF84FF0A0436365024BA36510BD00BF09
:1027A000703E0020D83B00080378012B70B5054629
:1027B00050D12A4B446D98421BD1294B5A6B42F0A1
:1027C00080025A635A6D42F080025A655A6D5A6906
:1027D00042F080025A615A6922F080025A610E2149
:1027E00043205B69FEF7ACFC1E4BE3601E4BC4F854
:1027F00000380023C4F8003EC02323606E6D4FF400
:102800000413A3633369002BFCDA012333610C202A
:1028100000F024FE3369DB07FCD4122000F01EFE1A
:102820003369002BFCDA0026A6602846FFF740FF3C
:102830006B68C4F81068DB68C4F81468C4F81C68D6
:102840004BB90A4BA3614FF0FF336361A36843F0B8
:102850000103A36070BD064BF4E700BF703E00208B
:10286000003802404014004003002002003C30C009
:10287000083C30C0F8B5446D054600212046FFF7FE
:1028800035FFA96D00234FF001128F68C4F834386A
:102890004FF00066C4F81C284FF0FF3004EB4312E1
:1028A00001339F42C2F80069C2F8006BC2F8080900
:1028B000C2F8080BF2D20B686A6DEB6563621023F5
:1028C0001361166916F01006FBD1122000F0C6FD48
:1028D000D4F8003823F4FE63C4F80038A36943F445
:1028E000402343F01003A3610923C4F81038C4F84F
:1028F00014380A4BEB604FF0C043C4F8103B084B50
:10290000C4F8003BC4F81069C4F80039EB6D03F15A
:10291000100243F48013EA65A362F8BDB43B0008DB
:1029200040800010426D90F84E10D2F8003823F429
:10293000FE6343EA0113C2F8003870472DE9F04105
:102940000EB200EB86080D46D8F80C100F6807F0A1
:102950000303022B50D0032B50D03D4A3D4F012B97
:1029600018BF1746446D4FEA451E04EB0E030022C4
:10297000C3F8102B8A6905F1100C002A40D04A8A4E
:1029800005F158035B013A43E2500123D4F81C28B7
:1029900003FA0CF31343A6444A69C4F81C38002315
:1029A000CEF8103905F13F03002A39D00A8A898B05
:1029B0009208012988BF4A43C16D04EB830356186E
:1029C00041EA0242C66529465A602046FFF78EFE5C
:1029D000D8F80C301B8A43EA85531F4305F148039E
:1029E0005B01E7500123D4F81C2803FA05F51543D1
:1029F000C4F81C58BDE8F081174FB3E7174FB1E793
:102A000004EB4613D3F8002B22F40042C3F8002B4A
:102A1000D4F81C28012303FA0CF322EA0303BAE7D3
:102A200004EB83030E4A5A6004EB461629462046FF
:102A3000FFF75CFED6F8003923F40043C6F80039EE
:102A4000D4F81C38012202FA05F523EA0505CFE780
:102A500000800010008004100080081000800C101E
:102A600000040002826D1268C265FFF721BE0000FB
:102A70005831436D49015B5813F4004004D013F4FE
:102A8000001F14BF01200220704700004831436D31
:102A900049015B5813F4004004D013F4001F14BF25
:102AA000012002207047000000EB8101CB68196A09
:102AB0000B6813604B6853607047000000EB8103A4
:102AC00030B5DD68AA691368D36019B9402B84BF9B
:102AD000402313606B8A1468426D1C44013CB4FBB4
:102AE000F3F46343033323F0030302EB411043EA9F
:102AF000C44343F0C043C0F8103B2B6803F003030A
:102B0000012B09B20ED1D2F8083802EB411013F4B0
:102B1000807FD0F8003B14BF43F0805343F0005354
:102B2000C0F8003B02EB4112D2F8003B43F00443F3
:102B3000C2F8003B30BD00002DE9F041244D6E6D20
:102B400006EB40130446D3F8087BC3F8087B38072C
:102B50000AD5D6F81438190706D505EB84032146A3
:102B6000DB6828465B689847FA072FD5D6F81438F3
:102B7000DB072BD505EB8403D968CCB98B69488A70
:102B80005E68B6FBF0F200FB12628AB91868DA6878
:102B900090420DD2121A83E81400202383F3118887
:102BA0000B482146FFF78AFF84F31188BDE8F081C6
:102BB000012303FA04F26B8923EA02036B81CB68D9
:102BC00023B121460248BDE8F0411847BDE8F08135
:102BD000703E002000EB810370B5DD68436D6C69C9
:102BE0002668E6604A0156BB1A444FF40020C2F83A
:102BF00010092A6802F00302012A0AB20ED1D3F8A2
:102C0000080803EB421410F4807FD4F8000914BFC5
:102C100040F0805040F00050C4F8000903EB42122D
:102C2000D2F8000940F00440C2F80009D3F8340893
:102C3000012202FA01F10143C3F8341870BD19B939
:102C4000402E84BF4020206020682E8A841940F0E6
:102C50000050013C1A44B4FBF6F440EAC440C6E715
:102C6000F8B504461E48456D05EB4413D3F80869D2
:102C7000C3F80869F10717D5D5F81038DA0713D566
:102C800000EB8403D9684B691F68DA68974218D251
:102C9000D21B00271A605F60202383F3118821462E
:102CA000FFF798FF87F31188330617D5D5F8342836
:102CB0000123A340134211D02046BDE8F840FFF79E
:102CC0001FBD012303FA04F2038923EA02030381EF
:102CD0008B68002BE8D021469847E5E7F8BD00BF98
:102CE000703E002096482DE9F84F456D6E69AB693E
:102CF0001E4016F4805F6E61044605D0FEF722FE8A
:102D0000BDE8F84FFFF788BC002E12DAD5F8003E78
:102D10008B489B071EBFD5F8003E23F00303C5F880
:102D2000003ED5F8043823F00103C5F80438FEF757
:102D300033FE370502D58248FEF722FEB0040CD5DB
:102D4000D5F8083813F0060FEB6823F470530CBF66
:102D500043F4105343F4A053EB60310704D5636888
:102D6000DB680BB176489847F2025AD4B3020CD50F
:102D7000D4F85480DFF8C8A100274FF00109A36DF3
:102D80009B68F9B28B4280F08780F70619D5616D98
:102D90000A6AC2F30A1702F00F0302F4F012B2F546
:102DA000802F00F0A180B2F5402F0AD104EB8303FD
:102DB00001F58051DB68186A00231A469F4240F0F3
:102DC00087803003D5F8184813D5E10302D50020D9
:102DD000FFF7B2FEA20302D50120FFF7ADFE6303A9
:102DE00002D50220FFF7A8FE270302D50320FFF734
:102DF000A3FE750384D5E00702D50020FFF730FF5E
:102E0000A10702D50120FFF72BFF620702D50220A0
:102E1000FFF726FF23077FF573AF0320FFF720FF9F
:102E20006EE7D4F85480DFF818A100274FF00109AD
:102E3000A36D9B685FFA87FB5B4597D308EB4B1349
:102E4000D3F8002902F44022B2F5802F22D1D3F822
:102E50000029002A1EDAD3F8002942F09042C3F874
:102E60000029D3F80029002AFBDB5946606DFFF7E3
:102E70003DFC228909FA0BF322EA0303238104EBC8
:102E80008B03DB689B6813B15946504698475846F8
:102E9000FFF736FC0137CBE708EB4112D2F8003BD5
:102EA00003F44023B3F5802F10D1D2F8003B002B60
:102EB0000CDA628909FA01F322EA0303638104EB65
:102EC0008103DB68DB680BB150469847013756E752
:102ED0009C0708BF0A68072B98BF027003F1010323
:102EE0009CBF120A013069E7023304EB830201F54B
:102EF0008051526890690268D0F808C04068A2EB1F
:102F0000000E0022104697420AD104EB8304636846
:102F10009B699A683A449A605A6817445F6050E720
:102F200012F0030F08BF0868964588BF8CF80000B0
:102F300002F1010284BF000A0CF1010CE3E700BFBB
:102F4000703E0020436D03EB4111D1F8003B43F488
:102F50000013C1F8003B7047436D03EB4111D1F8FA
:102F6000003943F40013C1F800397047436D03EB97
:102F70004111D1F8003B23F40013C1F8003B704726
:102F8000436D03EB4111D1F8003923F40013C1F86C
:102F90000039704730B5039C0172043304FB0325EC
:102FA000C361049B03630021059B00604060C16016
:102FB000426102618561046242628162C16243636F
:102FC00030BD00000022416A41610161C26082623D
:102FD000C2626FF00101FEF7FFBF000003694269A2
:102FE000934203D1C2680AB100207047181D704790
:102FF00003691960C2680132C260C2691344826900
:103000000361934224BF436A03610021FEF7D8BFE6
:1030100038B504460D46E3683BB16269131D12687A
:10302000A3621344E362002038BD237A33B92946F2
:103030002046FEF7B5FF0028EDDA38BD6FF001003D
:10304000FBE70000C368C269013BC36043691344E6
:1030500082694361934224BF436A436100238362D0
:10306000036B03B11847704770B52023044683F300
:103070001188866A3EB9FFF7CBFF054618B186F383
:103080001188284670BDA36AE26A13F8015BA36247
:10309000934202D32046FFF7D5FF002383F3118824
:1030A000EFE700002DE9F84F04460E46904699469A
:1030B000202787F311880025AA46D4F828B0BBF151
:1030C000000F09D149462046FFF7A2FF20B18BF33C
:1030D00011882846BDE8F88FA16AE36AA8EB050BC2
:1030E0005B1A9B4528BF9B46BBF1400F1BD933465B
:1030F00001F1400251F8040B43F8040B9142F9D15D
:10310000A36A40334036A3624035A26AE36A9A421A
:1031100002D32046FFF796FF8AF311884545D8D29F
:1031200087F31188C9E730465A46FDF7F7FDA36AD1
:103130005B445E44A3625D44E7E7000010B5029C77
:103140000172043303FB0421C36100238362C36261
:10315000039B0363049B00604060C46042610261A2
:10316000816104624262436310BD0000026AC26072
:10317000426A4261026100228262C2626FF0010112
:10318000FEF72ABF436902699A4203D1C2680AB1B5
:1031900000207047184650F8043B0B607047000051
:1031A000C368C2690133C3604369134482694361E0
:1031B000934224BF436A43610021FEF701BF000030
:1031C00038B504460D46E3683BB123691A1DA26277
:1031D000E2691344E362002038BD237A33B92946FB
:1031E0002046FEF7DDFE0028EDDA38BD6FF0010065
:1031F000FBE7000003691960C268013AC260C26956
:10320000134482690361934224BF436A036100232C
:103210008362036B03B118477047000070B5202329
:1032200004460E4683F31188856A35B91146FFF7C7
:10323000C7FF10B185F3118870BDA36A1E70A36A21
:10324000E26A01339342A36204D3E1692046043960
:10325000FFF7D0FF002080F3118870BD2DE9F84FF3
:1032600004460D4691469A464FF0200888F311888F
:103270000026B346A76A4FB951462046FFF7A0FF84
:1032800020B187F311883046BDE8F88FA06AE76A5D
:10329000A9EB06033F1A9F4228BF1F46402F1BD9A8
:1032A00005F1400355F8042B40F8042B9D42F9D159
:1032B000A36A4033A3624036A26AE36A9A4204D307
:1032C000E16920460439FFF795FF8BF311884E45DD
:1032D000D9D288F31188CDE729463A46FDF71EFD7D
:1032E000A36A3B443D44A3623E44E5E70269436967
:1032F0009A4203D1C3681BB9184670470023FBE705
:10330000836A002BF8D0043B9B1AF5D01360C36886
:10331000013BC360C3691A44836902619A4224BFB6
:10332000436A0361002383620123E5E700F02EB9BD
:103330004FF08043002258631A610222DA6070471E
:103340004FF080430022DA60704700004FF0804366
:1033500058637047FEE7000010B5174CFEF726FDD6
:10336000FEF748FE802215492046FEF7CDFD0123D9
:1033700044F8180C0374124B124AD96821F4E06126
:103380000904090C0A431049DA60CA6842F08072E5
:10339000CA600E490A6842F001020A601022DA7718
:1033A000202283F82220002383F3118862B6084884
:1033B000BDE81040FEF7CABDFC360020E43B000823
:1033C00000ED00E00003FA05F0ED00E0001000E081
:1033D000EC3B00082DE9F84F1F4C4FF000086569E1
:1033E00004F11407C1464FF08043266A5B6AAA685D
:1033F0009E1B96421DD34FF0200AAA68236AD5F877
:103400000CB0134423622B68BB425F60A6EB02063C
:103410006361C5F80C8001D1FFF792FF89F3118831
:103420002869D8478AF311886569AB689E42E4D25F
:10343000D9E76269BA420CD0916823628E1B96600C
:10344000A86802282CBF1818981CBDE8F84FFFF791
:103450007DBFBDE8F88F00BFD4360020034B59680C
:103460005A68521A9042FBD8704700BF001000E023
:103470004B6843608B688360CB68C3600B694361B2
:103480004B6903628B6943620B68036070470000FD
:1034900008B5224B22481A6940F2FF110A431A610B
:1034A0001A6922F4FF7222F001021A611A691A6B7A
:1034B0000A431A631A6D0A431A651A4A1B6D1146AC
:1034C000FFF7D6FF184802F11C01FFF7D1FF17489C
:1034D00002F13801FFF7CCFF154802F15401FFF764
:1034E000C7FF144802F17001FFF7C2FF124802F152
:1034F0008C01FFF7BDFF114802F1A801FFF7B8FFEB
:103500000F4802F1C401FFF7B3FF0E4802F1E001DA
:10351000FFF7AEFFBDE8084000F0A2B80038024057
:10352000000002400C3C0008000402400008024079
:10353000000C02400010024000140240001802403B
:10354000001C02400020024008B500F0F9F9FFF726
:1035500003FFFFF73FF8BDE80840FEF7D3BE0000C9
:10356000704700004FF0804310B51A69920708D5E4
:1035700000241C61202383F31188FFF72BFF84F3C1
:103580001188BDE81040FFF747B80000104B1A6CD7
:1035900042F001021A641A6E42F001021A660D4AE4
:1035A0001B6E936843F0010393604FF080435322F6
:1035B0009A624FF0FF32DA6200229A615A63DA604F
:1035C0005A6001225A6108211A601C20FDF7B8BD1B
:1035D00000380240002004E01F4B1A696FEAC25213
:1035E0006FEAD2521A611A69C2F308021A614FF0E7
:1035F000FF301A695A69586100215A6959615A693C
:103600001A6A62F080521A621A6A02F080521A62D2
:103610001A6A5A6A58625A6A59625A6A1A6C42F0AD
:1036200080521A641A6E42F080521A661A6E0B4A61
:10363000106840F480701060186F00F44070B0F5AE
:10364000007F1EBF4FF4803018671967536823F45A
:103650000073536000F054B900380240007000401D
:10366000304B4FF080521A642F4A4FF440411160A2
:103670001A6842F001021A601A689207FCD59A682B
:1036800022F003029A60274B19469A6812F00C0246
:10369000FBD1186800F0F90018609A601A6842F4CB
:1036A00080321A600B689B03FCD54B6F43F001031B
:1036B0004B671C4B5A6F9007FCD51C4A5A601A681E
:1036C00042F080721A60184A53685904FCD5154BB1
:1036D0001A689201FCD5164A9A60164B1A68164B66
:1036E0009A42164B1BD1164A1168164A914216D1BE
:1036F00040F205121A600B4B9A6842F002029A607F
:103700009A6802F00C02082AFAD15A6C42F48042FC
:103710005A645A6E42F480425A665B6E704740F2B9
:103720000572E7E700380240007000400854400787
:1037300000948838002004E011640020003C02401E
:1037400000ED00E041C20F41084A08B55369116815
:103750000B4003F00103536123B1054A13680BB119
:1037600050689847BDE80840FEF756BF003C01404E
:10377000E0400020084A08B5536911680B4003F087
:103780000203536123B1054A93680BB1D06898478F
:10379000BDE80840FEF740BF003C0140E04000208B
:1037A000084A08B5536911680B4003F004035361DC
:1037B00023B1054A13690BB150699847BDE8084029
:1037C000FEF72ABF003C0140E0400020084A08B54F
:1037D000536911680B4003F00803536123B1054A94
:1037E00093690BB1D0699847BDE80840FEF714BF54
:1037F000003C0140E0400020084A08B553691168C8
:103800000B4003F01003536123B1054A136A0BB157
:10381000506A9847BDE80840FEF7FEBE003C0140F4
:10382000E0400020174B10B55C691A68144004F49E
:1038300078725A61A30604D5134A936A0BB1D06A11
:103840009847600604D5104A136B0BB1506B98472C
:10385000210604D50C4A936B0BB1D06B9847E20557
:1038600004D5094A136C0BB1506C9847A30504D5D5
:10387000054A936C0BB1D06C9847BDE81040FEF739
:10388000CBBE00BF003C0140E04000201A4B10B509
:103890005C691A68144004F47C425A61620504D5DC
:1038A000164A136D0BB1506D9847230504D5134A82
:1038B000936D0BB1D06D9847E00404D50F4A136E99
:1038C0000BB1506E9847A10404D50C4A936E0BB10E
:1038D000D06E9847620404D5084A136F0BB1506F3D
:1038E0009847230404D5054A936F0BB1D06F9847CE
:1038F000BDE81040FEF790BE003C0140E0400020D3
:10390000062108B50846FDF71BFC06210720FDF738
:1039100017FC06210820FDF713FC06210920FDF7FE
:103920000FFC06210A20FDF70BFC06211720FDF7EE
:1039300007FC06212820BDE80840FDF701BC000077
:1039400008B5FFF749FE00F00DF8FDF79FFDFDF704
:103950008BFFFDF75FFEFFF703FEBDE80840FFF7B2
:10396000E5BC0000002304491A465A50C818083321
:10397000802B4260F9D17047E0400020034611F8E7
:10398000012B03F8012B002AF9D1704712101213F2
:103990001211000053544D3332463F3F3F000000A8
:1039A00000000000943900083F00000013040000EC
:1039B000E03900083F00000019040000EA3900085F
:1039C0003F00000021040000F43900083F0000001F
:1039D000143700209C290020042E00206C32002087
:1039E00053544D3332463430780053544D333246BD
:1039F0003432780053544D333246343436585800FC
:103A00000096000000000000000000000000000020
:103A100000000000000000005514000841140008D8
:103A20007D1400086914000875140008611400086A
:103A30004D14000839140008891400080000000023
:103A40008D15000879150008B5150008A1150008A6
:103A5000AD150008991500088515000871150008B6
:103A60001116000800000000010000000000000026
:103A70000200000000000000B9170008211800082B
:103A800040004000AC3B0020BC3B00200200000096
:103A9000000000000300000000000000651800089E
:103AA0000000000010000000CC3B002000000000DF
:103AB0000100000000000000703E00200101020033
:103AC00025424F41524425002553455249414C253A
:103AD000004633354C696768746E696E6700303133
:103AE0003233343536373839414243444546000095
:103AF0004172647550696C6F740025424F415244A5
:103B0000252D424C00000000A522000811210008CC
:103B1000251700088922000843000000203B000808
:103B200009024300020100C0320904000001020240
:103B300001000524001001052401000104240202F3
:103B40000524060001070582030800FF090401009F
:103B5000020A00000007050102400000070581027B
:103B600040000000120000006C3B00081201100130
:103B700002000040830440570002010203010000DC
:103B80000403090400400000004000000040000061
:103B900000400000000001000000020000000200E0
:103BA000000002000000020000000200000002000D
:103BB0000000020000000000AD1900088D1C000884
:103BC000391D000840004000D03E0020D03E0020BB
:103BD00001000000E03E00208000000040010000E5
:103BE000030000006D61696E00000000043C0008E5
:103BF000E83E0020E04000200100000055330008AE
:103C00000000000069646C6500000000A000A802CC
:103C100000000000AAAAAAAA50001400FFFF00009A
:103C20000077000070A70A000000000000000000FC
:103C3000AAAAAAAA00000000FFFF000000000000DE
:103C4000000000000000100200000000AAAAAAAABA
:103C500000000001FFFB0000000000000000080061
:103C60002000000000000000AAAAAAAA100000007C
:103C7000FFFF00000008000000000000000000003E
:103C800000000000AAAAAAAA00000000FFFF00008E
:103C90000000000000000000000000000000000024
:103CA000AAAAAAAA00000000FFFF0000000000006E
:103CB000000000000000000000000000AAAAAAAA5C
:103CC00000000000FFFF00000000000000000000F6
:103CD00000000000000000000A00000000000000DA
:103CE00003000000000000000000000000000000D1
:103CF00000000000000000000000000000000000C4
:103D00000000000000000000FF0096000000000816
:103D100004000000803B00080000000000000000DC
:103D20000000000000000000000000000000000093
:00000001FF
